:020000040800F2
:1000000000C00120E9360008353700083537000800
:100010003537000835370008353700080000000084
:10002000000000000000000000000000353700085C
:100030003537000800000000353700080D070008BC
:1000400035370008353700083537000835370008E0
:1000500035370008353700083537000835370008D0
:1000600035370008353700083537000835370008C0
:1000700035370008353700083537000835370008B0
:1000800035370008353700083537000835370008A0
:100090003537000835370008353700083537000890
:1000A0003537000835370008353700083537000880
:1000B0003537000835370008353700083537000870
:1000C0003537000835370008353700083537000860
:1000D0003537000835370008353700083537000850
:1000E0003537000835370008353700083537000840
:1000F0003537000835370008353700083537000830
:10010000353700083537000835370008353700081F
:10011000353700083537000835370008353700080F
:1001200035370008353700083537000835370008FF
:1001300035370008000000000000000035370008D7
:10014000353700083537000835370008ED06000858
:1001500035370008353700083537000835370008CF
:1001600035370008353700083537000835370008BF
:100170003537000835370008000000000000000097
:10018000353700083537000808B1022070470020D5
:10019000704700BF30B94FF480330B604FF40073E9
:1001A000138070470220704708B10220704700207A
:1001B000704700BF08B1022070470020704700BFA1
:1001C00090B910B400240BE0002041F8040B043275
:1001D00092B200E00022B2F5007FF5D30134A4B260
:1001E0009C42F7D3002002E0FF2040B2704740B2AB
:1001F0005DF8044B704700BF08B1FF2000E000200D
:1002000040B270470020704712230B8000487047AF
:100210004000002004230B80004870473C00002071
:1002200010B50A46034C0448214600F04DFD204617
:1002300010BD00BF74010020EC38000810B50A465C
:10024000034C0448214600F03FFD204610BD00BF8E
:10025000740100200039000808B50A4620B9054895
:10026000054900F031FD03E00248034900F02CFD90
:10027000014808BD143900087401002008B50A4679
:1002800020B90548054900F01FFD03E00248034975
:1002900000F01AFD014808BD24390008740100204F
:1002A00008B50A4620B90548054900F00DFD03E0F0
:1002B0000248034900F008FD014808BD3039000834
:1002C000740100200368B3F1A04F22D130B587B08C
:1002D000104B5A6B42F080025A635A6C42F48042CF
:1002E0005A644FF4C05301930223029300240394F1
:1002F00004940A250595084801A903F03BF843201A
:100300002946224603F03EF9432003F06DF907B079
:1003100030BD7047003802400000024008B5014679
:10032000D0F8AC0301F55F7100F024FD08BD00BFFB
:1003300008B5C1EBC1039B000344D0F8AC03D3F86C
:10034000E02100F045FD08BD08B5C1EBC1039B00ED
:100350000344D0F8AC03DA6B00F06AFD08BD00BFBF
:1003600008B5D0F8AC0300F0DDFD08BD10B50446BB
:10037000C3680BB9002100E00121D4F8AC0300F000
:10038000BDFDD4F8AC0300F099FD10BD10B50446D6
:10039000D0F8AC0300F0B6FD2268D2F8003E43F07E
:1003A0000103C2F8003E10BD08B50268D2F8003E55
:1003B00023F00103C2F8003ED0F8AC0300F0ACFD1E
:1003C00008BD00BF08B5D0F8AC0300F0B9FD08BD0A
:1003D00008B5D0F8AC0300F0B1FD08BD08B5D0F801
:1003E000AC0300F0AFFD08BD08B5D0F8AC0300F0D9
:1003F000ABFD08BD38B503782BBB144CC4F8AC0377
:10040000C0F820424FF0A04323600723636002231B
:10041000E360002525616561A361E5612562656290
:10042000A562E562204602F099FB2046802102F099
:1004300033FB20462946402202F00AFB20460121D8
:10044000802202F005FB002038BD00BF74030020AD
:1004500008B5D0F8200202F0EFFB002008BD00BF75
:1004600010B51446D0F820021A46234602F034FE96
:10047000002010BD08B5D0F8200202F061FE002077
:1004800008BD00BF08B5D0F8200202F057FF0020D9
:1004900008BD00BF08B5D0F8200202F0F1FE002030
:1004A00008BD00BF08B5D0F8200202F01BFF0020F5
:1004B00008BD00BFD0F8202211F0800F08D001F055
:1004C0007F03C3EBC3039B00134493F832007047D0
:1004D00001F07F01C1EBC1018900114491F8D601FF
:1004E000704700BF08B5D0F8200202F0E3FD0020FD
:1004F00008BD00BF08B5D0F8200202F08DFE002034
:1005000008BD00BF08B5D0F8200202F045FE00206B
:1005100008BD00BF08B5D0F8200202F073FE08BD88
:1005200010B5094C20460949002200F0EBFB20469B
:10053000074900F0FBFB2046064901F05BFA204624
:1005400000F0FCFB10BD00BF2407002020000020AD
:10055000A000002000000020F0B587B0224B1A6BED
:1005600042F001021A631A6B42F002021A631A6B1C
:1005700042F004021A631A6B42F008021A6341F651
:10058000FF730193002502950127039704950595B4
:10059000164801A902F0EEFE4FF6E77301931448E6
:1005A00001A902F0E7FE4FF6FF730193114C2046BC
:1005B00001A902F0DFFE104801A902F0DBFE1023C2
:1005C000019303230293204601A902F0D3FE4FF4C6
:1005D0008056019602970395204601A902F0CAFEB3
:1005E000A66107B0F0BD00BF003802400000024025
:1005F0000004024000080240000C024008B5044814
:10060000044B03600023437102F09AFF08BD00BF52
:10061000480900200030024008B50D480D4B03602A
:10062000002380F851304FF4827242608360C360CF
:10063000036143614FF480228261C36103624362BC
:100640004FF4005383620723C36201F0BBFE08BD71
:10065000500900200030014000B593B01B4A136CD4
:1006600043F080531364A2F5E432136823F440434B
:1006700043F40043136001230693079302230C9372
:100680004FF480030D9308230E934FF4A8730F9338
:10069000042310930723119306A801F0D3FE00B1A1
:1006A000FEE70D23019302210291002303934FF4EF
:1006B000A05304934FF48053059301A802F04AF825
:1006C00000B1FEE713B05DF804FB00BF0038024044
:1006D00008B502F0B3FFFFF7BFFFFFF73DFFFFF7DD
:1006E0008DFFFFF799FFFFF71BFFFEE710B5054CE5
:1006F0004FF08053A361044802F0B4FA4FF48053E2
:10070000A36110BD000802407403002008B502F088
:10071000AFFF08BD08B54FF0FF300221002202F004
:1007200031FF08BD0268044B9A4204D1034A136B9F
:1007300043F4805313637047003002400038024096
:1007400002680D4B9A4216D100B587B00B4A536C24
:1007500043F480535364F0230193022302930393E1
:100760000123049305230593054801A902F002FE25
:1007700007B05DF804FB70470030014000380240CC
:100780000000024038B50D4613460222C0F8F4219D
:100790008361C36100212A46FFF7ACFE002038BD0B
:1007A00010B50C46134600212246FFF7A3FE002099
:1007B00010BD00BF10B50C46134600212246FFF7BE
:1007C000A1FE002010BD00BF08B50423C0F8F4311D
:1007D00000210A460B46FFF78DFE002008BD00BF32
:1007E00008B50523C0F8F43100210A460B46FFF78F
:1007F00089FE002008BD00BF0346002002E0013052
:10080000C0B201331A78002AF9D170474B88012B06
:100810000BD110B50446C0F80432D0F814329B68EE
:1008200098472046FFF7D0FF10BD70470B78037044
:100830004B7843708B78CA7803EB022343800B79A3
:100840004A7903EB022383808B79CA7903EB022375
:10085000C380704710B504468021FFF71BFE204679
:100860000021FFF717FE10BD30B583B004460D46DA
:100870004A88130A013B062B00F28580DFE803F06B
:10088000040D238383657300D0F810321B68007C4D
:100890000DF106019847014679E0037C4BB9D0F889
:1008A00014329B6A0DF106009847014602234370FB
:1008B0006DE0D0F81432DB6A0DF10600984701466E
:1008C0000223437063E0D2B2052A3AD8DFE802F08F
:1008D000030C151E2730D0F810325B68007C0DF138
:1008E00006019847014652E0D0F810329B68007C20
:1008F0000DF106019847014649E0D0F81032DB6857
:10090000007C0DF106019847014640E0D0F8103216
:100910001B69007C0DF106019847014637E0D0F8CD
:1009200010325B69007C0DF10601984701462EE00C
:10093000D0F810329B69007C0DF106019847014602
:1009400025E02946FFF786FF2EE0037C3BB9D0F86F
:1009500014325B6B0DF106009847014617E02946FB
:10096000FFF778FF20E0037C4BB9D0F814321B6B03
:100970000DF10600984701460723437007E029461A
:10098000FFF768FF10E02946FFF764FF0CE0BDF8B1
:1009900006304BB1EA883AB19A4228BF1A46ADF800
:1009A00006202046FFF7EEFE03B030BD38B5044602
:1009B0008B88E3B9CB88D3B98D7805F07F0590F8A3
:1009C000FC31032B02D1FFF745FF38BD80F8FE5103
:1009D0002946FFF787FD2046FFF7F6FE1DB10223EB
:1009E00084F8FC3138BD012384F8FC3138BD204641
:1009F000FFF730FF38BD00BF38B504460D46897893
:100A0000264B1970012903D92946FFF723FF38BD6A
:100A100090F8FC31022B02D0032B15D039E081B1C4
:100A20004160032380F8FC3100F08EF9022804D1E4
:100A300020462946FFF70EFF38BD2046FFF7C4FECB
:100A400038BDFFF7C1FE38BD49B9022380F8FC313B
:100A5000416000F087F92046FFF7B6FE38BD4368D5
:100A6000994213D0D9B200F07DF90C4B197861602E
:100A7000204600F069F9022804D120462946FFF7F4
:100A8000E9FE38BD2046FFF79FFE38BDFFF79CFE0C
:100A900038BD2946FFF7DEFE38BD00BF60010020EB
:100AA00008B50346CA88012A02D0FFF7D3FE08BD65
:100AB00090F8FC21022A02D0032A08D00CE001465B
:100AC000002241F8082F0122FFF75CFE08BD191D26
:100AD0000122FFF757FE08BDFFF7BCFE08BD00BFAF
:100AE00008B5034690F8FC21023A012A0DD80122EC
:100AF000C260D0F804220AB10322C260184603F192
:100B00000C010222FFF73EFE08BDFFF7A3FE08BD61
:100B100010B5044690F8FC31023B012B0DD84B88F0
:100B2000012B0CD10023C0F80432D0F814329B689A
:100B300098472046FFF748FE10BDFFF78BFE10BD1B
:100B400008B54B78092B1BD8DFE803F011171A14EE
:100B50001A08051A0E0BFFF787FE13E0FFF726FFB2
:100B600010E0FFF749FF0DE0FFF79AFF0AE0FFF7FB
:100B7000B7FF07E0FFF74AFE04E0FFF7C9FF01E017
:100B8000FFF768FE002008BD38B504460D4690F812
:100B9000FC31032B0FD10B79012B09D8D0F814327B
:100BA0009B689847EB8843B92046FFF70DFE04E0A9
:100BB000FFF750FE01E0FFF74DFE002038BD00BFFB
:100BC00038B505460C468A88D1B26378012B26D009
:100BD000002B48D0032B74D190F8FC31022B02D0AB
:100BE000032B07D017E000296BD0802969D0FFF7CD
:100BF00051FC66E0638823B919B1802901D0FFF761
:100C000049FCD5F814329B68284621469847284667
:100C1000FFF7DAFD55E02146FFF71CFE51E090F8A2
:100C2000FC31022B02D0032B07D018E0002948D05A
:100C3000802946D0FFF72EFC43E06388002B40D18B
:100C400011F07F0F07D0FFF72DFCD5F814329B6809
:100C50002846214698472846FFF7B6FD31E0214651
:100C6000FFF7F8FD2DE090F8FC31022B02D0032BAA
:100C700006D023E011F07F0F23D0FFF70BFC20E01C
:100C800012F0800F05D001F07F0400EB041414343F
:100C900005E001F07F0400EB041404F5827428469B
:100CA000FFF708FC10B10123236001E0002323605B
:100CB000284621460222FFF765FD02E02146FFF7A4
:100CC000C9FD002038BD00BFD0B170B50D46164635
:100CD0000446FFF791FD0130400080B2308028705B
:100CE00003236B70022307E05A1CD2B20134E9548B
:100CF000531CDBB20021A95421780029F4D170BD26
:100D0000704700BF80B108B503460020C3F8140245
:100D100009B1C3F81012012183F8FC111A701846AA
:100D2000FFF768FB002008BD0220704719B1C0F82A
:100D30001412002070470220704700BF08B5FFF76B
:100D400087FB002008BD00BF08B5D0F8143223B1DE
:100D50001B68984718B1022008BD022008BD00207A
:100D600008BD00BF08B5D0F814325B689847002072
:100D700008BD00BF38B5044600F502752846FFF7E8
:100D800055FD0123C4F8F431B4F80E32C4F8F8313B
:100D900094F8081201F01F03012B08D013B1022BA5
:100DA0000AD00EE020462946FFF7CAFE0EE0204694
:100DB0002946FFF7E9FE09E020462946FFF700FF34
:100DC00004E0204601F08001FFF764FB002038BDFD
:100DD00038B5044609BBD0F8F431032B26D1D0F83E
:100DE0000C31D0F810118B420AD95B1AC0F80C31C3
:100DF0008B4228BF0B4611469AB2FFF7DBFC15E089
:100E0000D0F814321B6923B190F8FC21032A00D1D9
:100E100098472046FFF7D8FC08E0D0F814329B69C9
:100E200023B190F8FC21032A00D19847002038BD57
:100E300038B50446B9BBD0F8F431022B2BD1C169C7
:100E4000036A994206D9CB1AC36111469AB2FFF7D9
:100E5000A7FC20E08169B1FBF3F203FB12126AB92F
:100E60008B420BD8D0F8F831994207D200210A46BC
:100E7000FFF796FC0023C4F8F8310CE0D4F81432E4
:100E8000DB682BB194F8FC21032A01D12046984756
:100E90002046FFF7A5FC94F80032012B0CD100236B
:100EA00084F8003208E0D0F814325B6923B190F87E
:100EB000FC21032A00D19847002038BD38B50446EC
:100EC00000210A464023FFF7CBFA4025C4F8105111
:100ED0002046802100222B46FFF7C2FA256201231B
:100EE00084F8FC31D4F818322BB1D4F814325B6892
:100EF000204621799847002038BD00BF01740020AA
:100F0000704700BF90F8FC3180F8FD31042380F871
:100F1000FC310020704700BF90F8FD3180F8FC31B3
:100F20000020704708B590F8FC31032B04D1D0F8AD
:100F30001432DB6903B19847002008BD00207047D8
:100F4000002070470020704708B5012280F8FC217E
:100F5000D0F81422526801799047002008BD00BFE4
:100F600010B4D0F81842537813F0010F0DD1D0F817
:100F70001C32D86901EBC1018900084401790531AF
:100F800013798B4203D90B4601E00723064863819E
:100F900004E0013B9BB2C15CE2181173002BF8D155
:100FA00000205DF8044B704740390008D0F8180263
:100FB0000823438105E0013B9BB2044AD15CC2187F
:100FC0001173002BF7D10020704700BF5039000883
:100FD000D0F818020823438105E0013B9BB2044A84
:100FE000D15CC2181173002BF7D10020704700BFED
:100FF0004839000810B4D0F81842002304E0E11882
:10100000002008730133DBB2112BF8D9702323734E
:101010000C23E37494F85C3294F85D128B4212D086
:1010200003F1470104EBC1010879A073487A2076E7
:10103000097A61760133DBB284F85C32042B02D189
:10104000002384F85C32122363811379122B00D8B9
:10105000638100205DF8044B704700BFD0F8183260
:1010600000205881704700BF10B4D0F8184294F89F
:101070005D1201F1470004EBC00002711B028360A6
:101080000131C9B284F85D12042902D1002384F829
:101090005D325DF8044B704770B50446D0F81852C5
:1010A000D5F814323BB195F8191205222023FFF729
:1010B000DBFFFF2313E00E46D0F81C329B68084686
:1010C0009847034648B12046314602223A23FFF7AB
:1010D000CBFF05232B72FF2301E000226A8158B267
:1010E00070BD00BF70B582B005460E46D0F81842FC
:1010F000002304E0E2180021117301339BB20B2B93
:10110000F8D9D5F81C325B68304669460DF1060205
:101110009847014638B12846314602223A23FFF764
:10112000A3FFFF2118E00823E373009A531E180E53
:101130002074C3F307406074C3F30723A374013A18
:10114000E27402232375BDF80630002262751A0A84
:10115000A275E3750C23638148B202B070BD00BF75
:10116000F8B505460F46D0F81842D0F81C325B6837
:10117000084604F5187104F25E22984738B12846F3
:10118000394602223A23FFF76FFFFF261DE006468D
:10119000B4F85E124FF4007393FBF1F3A4F86A32D3
:1011A000D4F86022531E180E2073C3F307406073F7
:1011B000C3F30723A373013AE27300232374637418
:1011C0000B0AA374E1740823638170B2F8BD00BFF9
:1011D00010B5D0F818421344D4F86042A34205D9A0
:1011E00005222123FFF740FFFF2000E0002040B24E
:1011F00010BD00BF2DE9F84307468946D0F81842D4
:10120000B4F86A52B4F868329D4228BF1D46B4F85B
:101210005E6206FB05F6D0F81C32D3F810C004F16C
:101220000C0808464146D4F864222B46E0470028C3
:1012300007DA3846494604221123FFF715FFFF203D
:101240001BE0384681214246B3B2FFF753F9D4F888
:1012500064322B44C4F86432B4F868325D1BADB21A
:10126000A4F86852D4F834329E1BC4F834621DB915
:1012700003232372002000E0002040B2BDE8F88381
:10128000F8B506460F46D0F81842237A002B47D10E
:10129000154694F91832002B07DB94F81912052231
:1012A0002023FFF7E1FEFF2043E0D0F81C329B68CB
:1012B0000846984738B13046394602223A23FFF7AC
:1012C000D3FEFF2035E0AA78EB781B0443EA0263E3
:1012D0002A7943EA02236A791A43C4F86422EB7933
:1012E000297A41EA0323A4F8683230463946FFF7E9
:1012F0006FFF00281CDB02232372D4F81422B4F8F9
:101300006812B4F85E3203FB01F39A4208D030460B
:1013100094F8191205222023FFF7A6FEFF2008E00B
:101320004FF40073638130463946FFF763FF00E0F6
:10133000FF2040B2F8BD00BF2DE9F04106468846C7
:10134000D0F81842B4F86852B5F5007F01D34FF4D5
:101350000075D6F81C32D3F814C004F10C07D4F889
:101360006422B4F85E3240463946B2FBF3F2B5FB74
:10137000F3F3E047002807DA30464146042203230E
:10138000FFF772FEFF2021E0D4F864322B44C4F84A
:101390006432B4F868325B1B9BB2A4F86832D4F8AC
:1013A0003422551BC4F834522BB93046002100F0CA
:1013B0007BF900200AE0304601213A46B3F5007F70
:1013C00028BF4FF40073FFF79DF8002040B2BDE83E
:1013D000F08100BF2DE9F04105460F46D0F81842D4
:1013E000237A002B6ED1164694F91832002B08DAB6
:1013F00094F8191205222023FFF736FE4FF0FF085C
:1014000066E0D0F81C329B680846984740B12846F1
:10141000394602223A23FFF727FE4FF0FF0857E034
:10142000D5F81C32DB6838469847804640B12846DC
:10143000394602222723FFF717FE4FF0FF0847E047
:10144000B278F3781B0443EA0263327943EA022359
:1014500072791A43C4F86422F379317A41EA03239A
:10146000A4F8683228463946FFF7B2FE00282DDB83
:10147000B4F85E12D4F8642201FB02F2C4F86422CC
:10148000B4F8683203FB01F39BB2A4F86832D4F8D5
:1014900014229A4209D0284694F8191205222023D2
:1014A000FFF7E2FD4FF0FF0812E00121217228460C
:1014B00004F10C02B3F5007F28BF4FF40073FFF76F
:1014C00021F805E0FFF738FF804601E04FF0FF0804
:1014D0004FFA88F0BDE8F08110B5D0F81842537883
:1014E00013F0020F05D005222423FFF7BDFDFF20D6
:1014F0000BE0D4F86422B4F86832FFF769FE0028E4
:1015000002DB0020608100E0FF2040B210BD00BF80
:1015100008B513785A2B53D8DFE803F02E52523116
:1015200052525252525252525252525252523452B9
:101530005252525252523D3752523A5252525243E2
:101540005246525249524C525252524F5252525299
:10155000525252525252525252525252525252526B
:10156000525252525252525252525252525252525B
:101570005252525252524000FFF78EFD25E0FFF7C3
:1015800039FD22E0FFF7ECFC1FE0FFF767FD1CE0F0
:10159000FFF764FD19E0FFF709FD16E0FFF718FDFE
:1015A00013E0FFF79FFD10E0FFF7DAFD0DE0FFF716
:1015B00067FE0AE0FFF70EFF07E0FFF78DFF04E08C
:1015C00005222023FFF750FDFF2040B208BD00BFD9
:1015D00038B50546D0F8184294F818323BB9D4F81B
:1015E000143223B1637A13B90121FEF753FF284661
:1015F0008121FEF74FFF637A022B06D12846012195
:1016000004F503721F23FEF77DFF38BD10B50C46AD
:10161000D0F81812D1F814329A4228BF1A4693B261
:10162000D1F83422D21AC1F83422002281F83822AB
:1016300004220A7281212246FEF75CFF10BD00BF22
:1016400038B50546D0F8184200202072607284F840
:101650005D0284F85C02D5F81C321B689847284666
:101660000121FEF70FFF28468121FEF70BFF2846D8
:10167000012104F503721F23FEF744FF38BD00BFAC
:1016800008B5D0F81822002313720121517202F517
:1016900003721F23FEF736FF08BD00BFD0F81832D3
:1016A00000221A72704700BF38B50546D0F81842BC
:1016B0000A4BC4F82C3284F838120023237281219B
:1016C00004F50B720D23FEF715FF2846012104F5E2
:1016D00003721F23FEF716FF38BD00BF5553425358
:1016E00010B50446D0F81822137A022B03D012D377
:1016F000042B0DD910BD92F8191202F21B22FFF72C
:1017000007FF002807DA20460121FFF7CDFF10BDB3
:101710000021FFF7C9FF10BD38B50546D0F81842C3
:10172000D4F81032C4F83032D4F81432C4F8343259
:101730000121FEF7EFFE1F280DD1D4F80C221F4B1C
:101740009A4208D194F81912012904D894F81A324F
:101750000BB1102B0CD9284694F81912052220231E
:10176000FFF782FC022363722846FFF731FF38BD82
:10177000284604F21B22FFF7CBFE00280BDA237A5F
:10178000052B04D128460121FFF78EFF38BD2846DE
:10179000FFF71EFF38BD237A013BDBB2022B0CD9C9
:1017A00062892AB1284604F10C01FFF72FFF38BDEA
:1017B0001AB928460021FFF777FF38BD5553424339
:1017C00010B50446D0F81822137A13B1012B03D0B8
:1017D00010BDFFF7A1FF10BD92F8191202F21B22F3
:1017E000FFF796FE002803DA20460121FFF75CFF91
:1017F00010BD00BF10B5D0F81842637A022B05D196
:101800008121FEF747FE0023637210BD11F0800FA7
:1018100004D0012B02D00121FFF746FF10BD00BF0D
:10182000202303800048704780000020202303808D
:1018300000487047D80000202023038000487047EC
:10184000540000200A2303800048704774000020E1
:1018500010B50446037C6BB9012102224FF40073DA
:10186000FEF7FEFD2046812102224FF40073FEF7B1
:10187000F7FD0AE0012102224023FEF7F1FD204698
:10188000812102224023FEF7EBFD4FF41B7001F093
:1018900053FFC4F8180220B12046FFF7D1FE002004
:1018A00010BD012010BD00BF10B504460121FEF798
:1018B000E1FD20468121FEF7DDFD2046FFF7EEFE2B
:1018C000D4F8180220B101F03FFF0023C4F8183209
:1018D000002010BDF8B506460C46D0F818720B78FB
:1018E00013F0600536D0202D75D14A78FE2A02D03B
:1018F000FF2A1AD02AE04A888AB9CA88012A0ED15A
:1019000013F0800F0BD0D0F81C329B6998473860D9
:10191000304639460122FEF735FF00255CE03046AF
:101920002146FEF797FF022556E04A8842B9CA8849
:1019300032B913F0800F03D1FFF7A2FE00254BE070
:1019400030462146FEF786FF022545E0FEF782FF7E
:10195000022541E04B780A2B04D00B2B07D0012B3A
:101960003AD107E0391D0122FEF70CFF34E08B78F5
:101970007B6031E00979FEF785FD30462179FEF77D
:1019800079FD94F90430002B10DA337C3BB93046F2
:10199000812102224FF40073FEF762FD16E030460B
:1019A000812102224023FEF75BFD0FE0337C3BB92F
:1019B0003046012102224FF40073FEF751FD05E08D
:1019C0003046012102224023FEF74AFD30462179AC
:1019D000FFF710FF00E000252846F8BD08B5FFF727
:1019E0007FFE002008BD00BF08B5FFF7E9FE00201C
:1019F00008BD00BF09B1C0F81C120020704700BF2D
:101A00000C4B01E0013B10D00269002AFADA0369AD
:101A100043F001030361074B01E0013B07D002697A
:101A200012F0010FF9D10020704703207047032006
:101A3000704700BF400D030084B010B5044603A8F2
:101A400080E80E00089B012B18D1A36B23F4803390
:101A5000A363E36823F4840323F04003E360E368B3
:101A600023F44013E3600D9B012B03D1E36843F49F
:101A70008013E3602046FFF7C3FF09E0E36843F00B
:101A80004003E3602046FFF7BBFF4FF48033A363BE
:101A9000069B012B07D1A36843F00C03A360A36846
:101AA00043F02003A3600020BDE8104004B070475D
:101AB000836843F00103836000207047836823F04C
:101AC000010383600020704708B5C36823F0C0435A
:101AD000C360012904D1C36843F00053C36004E02C
:101AE00019B9C36843F08043C360322001F0CEFDD2
:101AF000002008BD490141F020010161054B01E0D2
:101B0000013B05D0026912F0200FF9D10020704787
:101B100003207047400D030010230361054B01E0D3
:101B2000013B05D0026912F0100FF9D10020704777
:101B300003207047400D0300D0F800381943C0F867
:101B400000180020704700BF84B0F8B5044607A80D
:101B500080E80E00A36B43F40023A3630F9E1EB91D
:101B6000A36B43F40013A3630023C4F8003E04F501
:101B70000065D4F80038C4F800380C9B012B0BD159
:101B8000099B23B920460021FFF7D6FF08E0204635
:101B90000121FFF7D1FF03E020460321FFF7CCFF2F
:101BA00020461021FFF7A6FF2046FFF7B5FF0023D0
:101BB0002B616B614FF0FF32AA61EB61079848B36C
:101BC00004F51063002219461F68002F03DA4FF056
:101BD00090471F6001E000271F6000270F61FF276B
:101BE0008F60013220338242EDD304F5306300224E
:101BF00019461F68002F03DA4FF090471F6001E07D
:101C000000271F6000270F61FF278F6001322033FC
:101C10008242EDD12B6923F480732B610A9B012B47
:101C20000ED1184B2B632B6B43F4803343F003032B
:101C30002B632B6B0023A3616FF08043636109E08A
:101C40000022A2616FF0804262611BB9A36943F078
:101C50001003A361A2690C4B1343A3610D9B1BB13D
:101C6000A36943F00803A361012E05D1A36943F0E2
:101C7000804343F00403A3610020BDE8F84004B0B2
:101C8000704700BF0001800000383C80D0F8083861
:101C900000F5006013F0060F10D0836803F0060310
:101CA000022B0DD0836803F00603062B0AD083684D
:101CB00003F00603042B07D1022070470020704771
:101CC00003207047032070470020704770B44B78A2
:101CD000012B1FD1D0F81C280D78AB409BB21343C9
:101CE000C0F81C380E78730103F510631A5812F40B
:101CF000004F2DD11C5844F0805545F400458A68AA
:101D0000C2F30A042C43CA7844EA824242EA865269
:101D10001A501DE0D0F81C280D784FF48033AB40EA
:101D20001343C0F81C380B785B0103F530631A5875
:101D300012F4004F0CD11A5842F0805444F400447D
:101D40008A68C2F30A022243C97842EA81421A50E1
:101D5000002070BC704700BF30B44B78012B1BD102
:101D6000D0F83C580C7803FA04F4A4B225EA040431
:101D7000C0F83C48D0F81C480D78AB409BB224EA30
:101D80000303C0F81C380B785B0103F510631A5885
:101D900022F400421A5019E0D0F83C480D78012294
:101DA00002FA05F524EA0544C0F83C48D0F81C487E
:101DB0000D78AA4024EA0242C0F81C280B785B0187
:101DC00003F530631A5822F400421A50002030BC48
:101DD000704700BF30B44B78012B68D14B69EBB929
:101DE0000B7800EB4313D3F8104924F0FF5424F48C
:101DF000C014C3F810490B7800EB4313D3F8104913
:101E000044F40024C3F810490B7800EB4313D3F8D3
:101E10001049E40CE404C3F810492CE00B7800EB03
:101E20004313D3F81049E40CE404C3F810490B78C9
:101E300000EB4313D3F8104924F0FF5424F4C014EA
:101E4000C3F810498B684C699C4200D94B610B78F0
:101E500000EB4313D3F8104944F40024C3F81049AD
:101E60000B7800EB4313D3F810594C69C4F31204F8
:101E70002C43C3F81049012A06D10B7800EB431319
:101E80000A69C3F8142909E04B693BB1D0F834283A
:101E90000D780123AB401343C0F834380B785B0155
:101EA00003F51063C25842F00442C2503BE00B7885
:101EB00000EB4313D3F8104BE40CE404C3F8104BCD
:101EC0000B7800EB4313D3F8104B24F0FF5424F4A9
:101ED000C014C3F8104B4B690BB18B684B610B7886
:101EE00000EB4313D3F8104B44F40024C3F8104B19
:101EF0000B7800EB4313D3F8105B8C68C4F3120427
:101F00002C43C3F8104B012A05D10B7800EB431387
:101F1000CA68C3F8142B0B785B0103F53063C25811
:101F200042F00442C250002030BC704730B49DF8EB
:101F3000084064B903339B1009D000F5805000EBD2
:101F4000023251F8045B15600134A342F9D100203C
:101F500030BC704770B582B04B78012B40F0A9803F
:101F60004B69EBB90B7800EB4313D3F8104924F01D
:101F7000FF5424F4C014C3F810490B7800EB43134A
:101F8000D3F8104944F40024C3F810490B7800EB4F
:101F90004313D3F81049E40CE404C3F8104945E0B6
:101FA0000B7800EB4313D3F81049E40CE404C3F8B6
:101FB00010490B7800EB4313D3F8104924F0FF5479
:101FC00024F4C014C3F810490C7800EB4414D4F87E
:101FD00010598E684B693344013BB3FBF6F3724EE4
:101FE00006EAC3432B43C4F810390B7800EB4313C4
:101FF000D3F810594C69C4F312042C43C3F81049A8
:10200000CB78012B40F0C8800B7800EB4313D3F85A
:10201000104924F0C044C3F810490B7800EB431377
:10202000D3F8104944F00054C3F81049012A06D1EE
:102030000B7800EB43130C69C3F814490CE0CB7820
:10204000012B0CD04B6903B3D0F834480E78012330
:10205000B3402343C0F83438CB78012B15D1D0F8E6
:10206000083813F4807F08D10B785B0103F5106307
:10207000C45844F00054C45007E00B785B0103F5EA
:102080001063C45844F08054C4500B785B0103F5CE
:102090001063C45844F00444C450CB78012B7FD162
:1020A00014460B46C9681A789B8A0094FFF73EFFD6
:1020B00076E00B7800EB4313D3F8104BE40CE40408
:1020C000C3F8104B0B7800EB4313D3F8104B24F0FC
:1020D000FF5424F4C014C3F8104B4B69A3B90B7818
:1020E00000EB4313D3F8105B8C68C4F312042C4349
:1020F000C3F8104B0B7800EB4313D3F8104B44F4A8
:102100000024C3F8104B1DE08D680C7800EB4414DC
:10211000D4F8106B2B44013BB3FBF5F39BB2224D7B
:1021200005EAC3453543C4F8105B0C7800EB441452
:10213000D4F8106B8D6805FB03F3C3F3120333432C
:10214000C4F8103B012A05D10B7800EB4313CA6891
:10215000C3F8142BCB78012B15D1D0F8083813F421
:10216000807F08D10B785B0103F53063C25842F0E1
:102170000052C25007E00B785B0103F53063C25890
:1021800042F08052C2500B785B0103F53063C258B5
:1021900042F00442C25003E0012A7FF453AF47E704
:1021A000002002B070BD00BF0000F81F0332921083
:1021B0000FD030B40C46002300F580552D6844F84C
:1021C000045B01339A42F7D101EB8201084630BC2F
:1021D00070470846704700BF4B78012B13D10B782E
:1021E0005B0103F51063C258002A03DBC25822F0DA
:1021F0008042C2500B785B0103F51063C25842F471
:102200000012C25012E00B785B0103F53063C25834
:10221000002A03DBC25822F08042C2500B785B01D7
:1022200003F53063C25842F40012C25000207047D8
:102230004B78012B15D10B785B0103F51063C25865
:1022400022F40012C250CB78023BDBB2012B1DD826
:102250000B785B0103F51063C25842F08052C25004
:1022600014E00B785B0103F53063C25822F40012CE
:10227000C250CB78023BDBB2012B07D80B785B0155
:1022800003F53063C25842F08052C25000207047BC
:10229000D0F8003823F4FE63C0F80038D0F80038D6
:1022A000090101F4FE610B43C0F8003800207047BB
:1022B00008B5D0F8043823F00203C0F8043803202E
:1022C00001F0E4F9002008BD08B5D0F8043843F067
:1022D0000203C0F80438032001F0D8F9002008BD3B
:1022E0004369806918407047D0F8183800F50060DD
:1022F000C0691840000C704700F50063D0F818085A
:10230000DB69184080B2704700F5306303EB411180
:102310008B6800F5006040691840704710B4D0F831
:102320001048D0F8343800EB4110D0F80809CB4001
:10233000DB01DBB2234318405DF8044B704700BF5C
:10234000406900F001007047D0F8003923F4FF63C2
:1023500023F00703C0F8003900F500639A6802F023
:102360000602042A05D1D0F8002942F00302C0F881
:1023700000295A6842F480725A600020704700BFFA
:1023800010B40024C0F8104BD0F8104B44F40024D3
:10239000C0F8104BD0F8104B44F01804C0F8104BA4
:1023A000D0F8104B44F0C044C0F8104B012905D1BF
:1023B000C0F8142B4FF08023C0F8003B00205DF8DC
:1023C000044B704700283AD010B5044690F85130BD
:1023D00013F0FF0F01D1FEF7B3F9022384F8513057
:1023E0002268136823F04003136021686268A368C1
:1023F0001A43E3681A4323691A4363691A43A369BA
:1024000003F400731343E2691343226A1343A26A7D
:102410001A430A602168638B03F00402636A134362
:102420004B602368E26A1A612268D36923F400636F
:10243000D36100206065012384F8513010BD012074
:10244000704700BF38B50446036813F0010F3AD057
:10245000B34B9B6803F00C03042B00F04B81B04B93
:102460009B6803F00C03082B05D1AD4B5B6813F49C
:10247000800F40F041810022AA4B1A7001F000F950
:10248000054606E001F0FCF8401BB0F5FA7F00F2CB
:102490003581A34B1B6813F4003FF3D12279A14B84
:1024A0001A7063687BB101F0EBF8054606E001F0B5
:1024B000E7F8401BB0F5FA7F00F22281984B1B68C9
:1024C00013F4003FF3D0236813F0020F49D0944B6C
:1024D0009B6813F00C0F0AD0914B9B6803F00C0320
:1024E000082B09D18E4B5B6813F4800F04D1E3688D
:1024F000012B40F0078126E0E36893B101228A4B6B
:102500001A6001F0BDF8054605E001F0B9F8401B7E
:10251000642800F2F980824B1B6813F0020FF4D09C
:1025200011E00022804B1A6001F0AAF8054605E090
:1025300001F0A6F8401B642800F2E880784B1B6885
:1025400013F0020FF4D17648026822F0F8012269F4
:10255000F82393FAA3F3B3FA83F3DBB29A400A4366
:102560000260236813F0080F26D0636993B101223B
:102570006E4B1A6001F084F8054605E001F080F822
:10258000401B642800F2C480654B5B6F13F0020FA0
:10259000F4D011E00022654B1A6001F071F8054695
:1025A00005E001F06DF8401B642800F2B3805C4B3D
:1025B0005B6F13F0020FF4D1236813F0040F42D0C5
:1025C000574A136C43F080531364A2F5E432136846
:1025D00043F48073136001F053F8054605E001F001
:1025E0004FF8401B642800F29780514B1B6813F48E
:1025F000807FF4D000224F4B1A7001F041F805465D
:1026000007E001F03DF8401B41F28833984200F2A8
:102610008580434B1B6F13F0020FF2D1227A454B9A
:102620001A70A3687BB101F02BF8054606E001F0B3
:1026300027F8401B41F2883398427FD8384B1B6FF4
:1026400013F0020FF3D0A369002B79D0344B9B68B1
:1026500003F00C03082B75D00022374B1A6001F0F1
:102660000FF8054604E001F00BF8401B64286BD816
:102670002B4B1B6813F0007FF5D1A369022B65D1AA
:10268000216A626A47F6C07393FAA3F3B3FA83F33D
:10269000DBB29A401143A36A5B08013B4FF440321E
:1026A00092FAA2F2B2FA82F2D2B293400B43E269FA
:1026B0001343E26A4FF0706191FAA1F1B1FA81F12E
:1026C000C9B28A40134343F00053154A53600122B4
:1026D000194B1A6000F0D4FF044604E000F0D0FF6C
:1026E000001B642834D80E4B1B6813F0007FF5D014
:1026F000002038BD012038BD012038BD032038BD81
:10270000032038BD012038BD032038BD032038BD6B
:10271000032038BD032038BD032038BD032038BD59
:10272000003802400238024000004742800E474213
:10273000007000407038024060004742032038BDFE
:10274000002038BD012038BD032038BD002038BD31
:10275000032038BD70B504460D46874B1B6803F057
:102760000F038B426BD2CAB2834B1A701B6803F003
:102770000F038B4240F0E480036813F0020F06D091
:102780007E498B6823F0F002836813438B602368D3
:1027900013F0010F00F0B8806268012A05D1774B71
:1027A0001B6813F4003F0ED1CCE0022A05D1734B15
:1027B0001B6813F0007F06D1C6E0704B1B6813F056
:1027C000020F00F0C3806D498B6823F003031343AD
:1027D0008B6000F055FF05466368012B0FD107E0C1
:1027E00000F04EFF401B41F28833984200F2B08067
:1027F000624B9B6803F00C03042BF1D184E0022BA5
:1028000017D107E000F03CFF401B41F288339842AB
:1028100000F2A080594B9B6803F00C03082BF1D108
:1028200072E000F02DFF401B41F28833984200F225
:102830009380524B9B6813F00C0FF2D164E0036855
:1028400013F0020F06D04D498B6823F0F002836825
:1028500013438B60236813F0010F4DD06268012A87
:1028600005D1464B1B6813F4003F0DD176E0022AD8
:1028700005D1424B1B6813F0007F05D170E03F4B40
:102880001B6813F0020F6DD03C498B6823F00303E3
:1028900013438B6000F0F4FE06466368012B0ED1F3
:1028A00006E000F0EDFE801B41F2883398425BD8D1
:1028B000324B9B6803F00C03042BF2D11CE0022B7B
:1028C00015D106E000F0DCFE801B41F2883398420F
:1028D0004CD82A4B9B6803F00C03082BF2D10BE079
:1028E00000F0CEFE801B41F28833984240D8234B43
:1028F0009B6813F00C0FF3D1EAB21F4B1A701B68E0
:1029000003F00F03AB4235D1236813F0040F06D058
:102910001A498B6823F4E052E36813438B60236801
:1029200013F0080F07D0154A936823F46043216918
:1029300043EAC1039360002000F072FE002070BDE6
:10294000012070BD012070BD012070BD012070BD4F
:10295000032070BD032070BD032070BD012070BD39
:10296000012070BD012070BD032070BD032070BD2B
:10297000032070BD012070BD003C024000380240C1
:10298000224B9B6803F00C03042B3DD0082B01D095
:102990001F4870471D4B586800F03F005B6813F4F8
:1029A000800F10D01B4BB3FBF0F3184A506847F66A
:1029B000C072104092FAA2F2B2FA82F2D2B2D040C1
:1029C00000FB03F30FE0124BB3FBF0F30F4A506828
:1029D00047F6C072104092FAA2F2B2FA82F2D2B274
:1029E000D04000FB03F3094A506800F440304FF434
:1029F000403292FAA2F2B2FA82F2D2B2D040013060
:102A00004000B3FBF0F070470248704700380240C6
:102A10000024F40000127A0008B5FFF7B1FF094B5B
:102A20009B6803F0F002F02393FAA3F3B3FA83F365
:102A3000DBB222FA03F3044AD35CD840034B18609C
:102A400008BD00BF0038024058390008F8000020D7
:102A500030B40468636A19B943EA0240A06218E01E
:102A60000D46A06A03EB1040002308E003F140018B
:102A700004EB8101496800EB11400133DBB2691EB0
:102A80008B42F3DB40EA024005F13F0104EB810198
:102A90004860002030BC70470368596200207047CE
:102AA0002DE9F04782B007460D46D0F80080CB00F4
:102AB0005B1A9B0003445E6C9A6CB61A9B6B9E4239
:102AC00000D91E4616F1030901D509F103094FEAA1
:102AD000A90921E05E1AC5EBC5039B003B449B6B33
:102AE0009E4200D91E4616F1030901D509F10309DA
:102AF0004FEAA909EC00641BA4003C44E16B3B7C59
:102B000000934046EAB2B3B2FFF710FAE36B3344E6
:102B1000E363A36C3344A364424608EB451303F517
:102B200010639B699BB24B4509D9EB005B1B9B0073
:102B30003B44996C5B6C994201D2002BCAD1002EA8
:102B400007DC0123AB40D2F8341821EA0303C2F8B2
:102B50003438002002B0BDE8F08700BF002866D0FE
:102B6000F0B589B00446032380F87933FDF7AAFB5A
:102B70002068FEF7A3FF254655F8107B6E460FCD63
:102B80000FC695E80F0086E80F00231D0ECB3846D0
:102B9000FEF752FF20680021FEF796FF002210E0AA
:102BA000D3009B1A9B002344012183F8311083F842
:102BB0003020DA86002183F833109963D963596491
:102BC00001320E2AECD9002218E0D3009B1A9B0098
:102BD0002344002183F8D51183F8D421DA8683F8C1
:102BE000D711C3F8DC11C3F8E011C3F8E81123686A
:102BF00002F1400003EB8003596001320E2AE4D950
:102C0000254655F8107B6E460FCD0FC695E80F0090
:102C100086E80F00231D0ECB3846FEF795FF0123F3
:102C200084F879332068FFF74FFB002001E0012092
:102C3000704709B0F0BD00BF90F87833012B0ED07B
:102C400010B50446012380F878330068FFF730FBA5
:102C50002068FEF72DFF002084F8780310BD0220C5
:102C6000704700BF2DE9F84F044606683046FFF76D
:102C700067FB002840F01B822068FFF731FB00282B
:102C800000F015822068FFF72BFB10F0020F02D036
:102C9000236802225A612068FFF722FB10F4002FFC
:102CA0005CD02068FFF720FB0746002553E017F0B3
:102CB000010F4ED05FFA85F920684946FFF724FBE3
:102CC000804610F0010F31D006EB45130122C3F806
:102CD000082B03F530632269012A12D1EA00521B46
:102CE0009200224402F5EC71D2F8DC011B69C3F3B7
:102CF0001203C01AC2F8EC01D2F8E0214B68134469
:102D00008B6020464946FDF713FB2369012B0DD14B
:102D100065B9C5EBC5039B002344D3F8E8312BB953
:102D20002068012104F55F72FFF72AFB18F0080FF5
:102D300007D02046FDF7F2FA06EB45130822C3F848
:102D4000082B18F0100F04D006EB45131022C3F81F
:102D5000082B01357F08002FA9D100E0002520684D
:102D6000FFF7BEFA10F4802F6BD02068FFF7C4FA8B
:102D70000746002563E017F0010F5ED05FFA85F982
:102D800020684946FFF7CAFA804610F0010F2DD09F
:102D9000012202FA05F0D6F8343823EA0003C6F817
:102DA000343806EB4513C3F808292369934209D147
:102DB000EB005B1B9B00234403F13802D96B9B6B38
:102DC0000B44536020464946FDF7BEFA2369012BA8
:102DD0000CD15DB9C5EBC5039B0023445B6C2BB9DB
:102DE0002068012104F55F72FFF7CAFA18F0080F96
:102DF00004D006EB45130822C3F8082918F0100F79
:102E000004D006EB45131022C3F8082918F0400F30
:102E100004D006EB45134022C3F8082918F0020F2E
:102E200004D006EB45130222C3F8082918F0800FDE
:102E300003D020462946FFF733FE01357F08002FD7
:102E400099D12068FFF74CFA00280CDAD6F804383C
:102E500023F00103C6F804382046FDF7A5FA2368DD
:102E60004FF000425A612068FFF73AFA10F4006F01
:102E70000BD0D6F8083813F0010F02D02046FDF72A
:102E800085FA23684FF400625A612068FFF728FA38
:102E900010F4805F4ED0374606F50068D8F804304D
:102EA00023F00103C8F8043020680021FEF722FE59
:102EB000002207E007EB4213FF21C3F80819C3F80B
:102EC000081B013263689342F4D84FF0FF33C8F80F
:102ED0001830D8F81C3043F00113C8F81C30A36A2E
:102EE00063B1D8F8843043F00B03C8F88430D8F8C5
:102EF000443043F00B03C8F844300BE0D8F81430EA
:102F000043F00B03C8F81430D8F8103043F00B032B
:102F1000C8F81030D6F8003823F4FE63C6F800383D
:102F20002068217C04F55F72FFF72AFA23684FF4CA
:102F300080525A612068FFF7D3F910F4005F26D061
:102F40002068FFF701FA2268D36823F47053D36036
:102F50002068FEF79BFE50B90023E3604FF4007336
:102F600063612268D36843F41053D36008E00323FD
:102F7000E360402363612268D36843F4A053D360C5
:102F80002046FDF7F3F923684FF400525A61206898
:102F9000FFF7A6F910F0100F42D02268936923F0D2
:102FA00010039361376A07F00F08C7F34343022BFE
:102FB0001CD147F6F0731F402DD03F094FEAC809D6
:102FC000C8EB090A4FEA8A0AA2443046DAF8E0114F
:102FD0003A46FFF7EBF8DAF8E0313B44CAF8E03163
:102FE000DAF8EC311F44CAF8EC7114E0062B12D168
:102FF000304604F55F710822FFF7D8F8C7F30A17C7
:103000004FEAC803C8EB030292002244D2F8EC3125
:103010003B44C2F8EC312268936943F0100393619A
:103020002068FFF75DF910F0080F05D02046FDF786
:1030300097F9236808225A612068FFF751F910F4C4
:10304000801F07D02046E9B2FDF7C2F923684FF48C
:1030500080125A612068FFF743F910F4001F07D06F
:103060002046E9B2FDF7AEF923684FF400125A6129
:103070002068FFF735F910F0804F06D02046FDF7A5
:10308000ADF923684FF080425A612068FFF728F9B4
:1030900010F0040F0BD023685D6815F0040F02D008
:1030A0002046FDF7A1F923685A6815435D60BDE825
:1030B000F88F00BF90F87833012B0BD010B5044681
:1030C000012380F878330068FFF7E2F8002084F8E5
:1030D000780310BD0220704738B50546C8B210F01D
:1030E000800F07D001F07F04C4EBC404A400303487
:1030F0002C4407E001F07F04C4EBC404A4002C447A
:1031000004F5EA7401F07F012170C0096070A260CB
:10311000E37000B1E180022B01D10023237195F807
:103120007833012B0AD0012385F8783328682146AB
:10313000FEF7CCFD002085F8780338BD022038BDAD
:1031400010B50446CAB212F0800F07D001F07F0319
:10315000C3EBC3039B003033034407E001F07F035C
:10316000C3EBC3039B00034403F5EA7301F07F0143
:103170001970D2095A7094F87823012A0AD00122D2
:1031800084F8782320681946FEF7E6FD002084F8CD
:10319000780310BD022010BD70B501F07F06F40069
:1031A000A51BAD00054405F5EA712C46C5F8E021E4
:1031B000C5F8E8310023C4F8EC3184F8D53184F83F
:1031C000D4610369012B05D1C6EBC604A4000444F5
:1031D000C4F8E42190F87823012A11D00446012292
:1031E00080F8782326B90068DAB2FEF7F3FD03E031
:1031F0000068DAB2FEF7AEFE002084F8780370BDF6
:10320000022070BD01F07F01C1EBC10189000844BB
:10321000B0F8EC01704700BF70B501F07F06F40014
:10322000A51BAD0030354119A41BA4000444E26382
:1032300063640023A364012384F8313084F8306090
:103240000369012B04D1C6EBC604A4000444226424
:1032500090F87823012A11D00446012280F87823BF
:1032600026B90068DAB2FEF7B5FD03E00068DAB20D
:10327000FEF770FE002084F8780370BD022070BD58
:1032800038B50446CAB212F0800F07D001F07F03B0
:10329000C3EBC3039B003033034405E0C1EBC10320
:1032A0009B00034403F5EA730120987001F07F0549
:1032B0001D70D2095A7094F87823824210D084F895
:1032C000780320681946FEF787FF2DB92068217C16
:1032D00004F55F72FFF754F8002084F8780338BDD6
:1032E000022038BD10B50446CAB212F0800F07D0D4
:1032F00001F07F03C3EBC3039B003033034405E0BD
:10330000C1EBC1039B00034403F5EA7300209870EE
:1033100001F07F011970D2095A7094F87823012ABC
:103320000AD0012284F8782320681946FEF780FF2E
:10333000002084F8780310BD022010BD90F8783387
:10334000012B14D010B50446012380F8783311F016
:10335000800F05D0006801F07F01FEF7CBFB02E093
:103360000068FEF7D9FB002084F8780310BD022026
:10337000704700BF2DE9F0410023D3E09C460122B5
:103380009A400C681440944240F0CB804D68022D66
:1033900001D0122D14D14FEAD30808F1080850F8D3
:1033A000287003F0070E4FEA8E0E0F2505FA0EF572
:1033B00027EA05060D6905FA0EF5354340F8285051
:1033C00006684FEA430E032505FA0EF5ED4305EABC
:1033D00006074E6806F0030606FA0EF63E43066040
:1033E0004E68771E012F03D9112E01D0122E12D153
:1033F000866805EA0607CE6806FA0EF63E43866042
:10340000476827EA02074E68C6F3001202FA0CF674
:1034100046EA07024260C2682A408D6805FA0EF546
:103420001543C5604A6812F0805F7AD0404D6A6CDF
:1034300042F480426A649A08961CA5F5803555F8D6
:10344000266003F00307BF000F25BD4026EA0506EE
:10345000384DA84231D005F58065A8422BD005F53E
:103460008065A84225D005F58065A8421FD005F5E6
:103470008065A84219D005F58065A84213D005F5EE
:103480008065A8420DD005F58065A84207D005F5F6
:103490008065A84201D1082510E009250EE0072526
:1034A0000CE006250AE0052508E0042506E00325D2
:1034B00004E0022502E0012500E00025BD4035437F
:1034C00002321D4E46F822501C4A1568E24302EAB9
:1034D00005064F6817F4803F01D044EA0506174DF2
:1034E0002E606D6802EA05064F6817F4003F01D0B0
:1034F00044EA0506114D6E60AD6802EA05064F68A4
:1035000017F4801F01D044EA05060C4DAE60ED684B
:103510002A404E6816F4001F01D044EA0502074C09
:10352000E26001330F2B7FF629AFBDE8F08100BFC9
:10353000003802400000024000380140003C0140D9
:1035400058B110B50446437913F0FF0F01D1FDF7D0
:10355000E9F801236371002010BD0120704700BF0E
:1035600000F00700064AD36823F4E0631B041B0C39
:1035700043EA002040F0BF6040F40030D060704764
:1035800000ED00E030B4164BDC68C4F30224C4F153
:103590000705042D28BF0425231D062B01D9033C54
:1035A00000E00024012303FA05F5013D2940A14074
:1035B000A340013B1A400A43002806DA00F00F003E
:1035C0001201D2B2074B1A5407E01201D2B200F135
:1035D000604000F5614080F8002330BC704700BFB8
:1035E00000ED00E014ED00E0410900F01F000123B0
:1035F0008340024A42F82130704700BF00E100E0FA
:103600000138B0F1807F06D2044B586000209860EA
:1036100007221A6070470120704700BF10E000E0E9
:1036200008B5FFF7F9F9044BA3FB00308009FFF759
:10363000E7FF002008BD00BFD34D621008B50B4B5B
:103640001A6842F400721A601A6842F480621A60C2
:103650001A6842F480721A600320FFF781FF00208D
:10366000FFF7DEFFFDF756F8002008BD003C0240E2
:10367000024A136801331360704700BF64010020E1
:10368000014B1868704700BF6401002010B582B07C
:103690000190FFF7F5FF0446FFF7F2FF001B019BC7
:1036A0009842F9D302B010BD0C4B1A6842F00102E7
:1036B0001A60002199601A6822F0847222F4803224
:1036C0001A60074A5A601A6822F480221A60D96088
:1036D0004FF00062034B9A60704700BF0038024011
:1036E0001030002400ED00E0DFF830D0002103E0CE
:1036F0000B4B5B58435004310A480B4B42189A421B
:10370000F6D30A4A02E0002342F8043B084B9A42EF
:10371000F9D3FFF7C9FFFCF7DBFF704700C00120BA
:103720006A390008000000206001002060010020CC
:10373000AC090020FEE70000024B0146186800F0CB
:103740004FB800BF5C010020024B0146186800F032
:1037500003B800BF5C01002030B500293CD051F80F
:10376000042C0B1F1D49002AB8BF9B180A680C4681
:1037700012B95A600B6030BD93420DD219685818C7
:10378000904201BF5A5852181A60426823605A602A
:1037900030BD994203D80A4651680029F9D114680E
:1037A00015199D420AD11B682344D0188842136022
:1037B00012D10868034413604B680CE002D90C2353
:1037C000036030BD1C681819884201BF0868496849
:1037D000001918605960536030BD00BF6C010020B3
:1037E00070B5CC1C24F0030408340C2C38BF0C2416
:1037F000002C064603DA0C233360002070BD8C4297
:10380000F9D3204A136810461946A1B10A68121B61
:103810000ED40B2A03D90A608B188C501FE08B4200
:103820000BBF5A684A6802605A6018BF0B4616E020
:103830000B464968E9E7144D2B681BB9304600F088
:1038400025F828603046214600F020F8421C034647
:10385000D1D0C51C25F0030585420AD11C6003F1B7
:103860000B001A1D20F00700821A0AD0514299500D
:1038700070BD3046E91A00F009F80130BBD02B4684
:10388000ECE770BD6C0100206801002038B5064CE3
:10389000002305460846236000F008F8431C02D1C7
:1038A000236803B12B6038BDA8090020044A0549EC
:1038B0001368002B08BF0B46184410601846704769
:1038C00070010020AC090020008002021F000000EF
:1038D00053544D202020202050726F647563742053
:1038E0002020202020202020302E303153544D33F2
:1038F00032204D6173732053746F726167650000ED
:1039000053544D6963726F656C656374726F6E6951
:10391000637300003030303030303030303031417F
:10392000000000004D534320436F6E66696700003E
:103930004D534320496E74657266616365000000F3
:10394000000000030080830000060000000000006B
:10395000000000000000000000000000010203045D
:0A39600001020304060708094300F2
:10396A008901000895010008A9010008B5010008AD
:10397A00C1010008F901000805020008C83800085A
:10398A0009020008150200083D0200082102000889
:10399A00590200087D020008A10200080403090474
:1039AA00120100020000004083042A5700020102AB
:1039BA000301000009072000010104C032090400C4
:1039CA0000020806500507058102400000070501AC
:1039DA00024000000A060002000000400100000048
:1039EA0009022000010104C032090400000208068D
:1039FA0050050705810200020007050102000200C6
:103A0A0051180008A9180008D5180008000000007D
:103A1A0000000000DD190008E91900080000000094
:103A2A000000000000000000211800082D180008FE
:103A3A00391800084518000809022000010104C0CD
:103A4A0032090400000208065005070581024000F9
:103A5A0000070501024000000024F40000000000F5
:103A6A00000000000000000000000000000000004C
:103A7A000000000000000000000000006839000893
:103A8A00000000000000000000000000000000002C
:103A9A00000000000000000000000000000000001C
:103AAA00000000000000000000000000000000000C
:103ABA00000000000000000000000000FC000020E0
:04000005080036E9D0
:00000001FF
